:020000021000EC
:10F8000011241FBE1CC0CF93DF93AC0120E030E079
:10F810002817390760F4A0EDB7E0C0E0D0E0CD01D3
:10F820000197F1F72F5F3F4F24173507C0F3DF91A2
:10F83000CF9108958CB95E9BFECF5E9A0895C0EE7D
:10F84000DFE0DEBFCDBFCC24DD2476012601370109
:10F85000C25EDE4F19821882CE51D1403324032D6F
:10F86000AA24BB248091640081608093640080910D
:10F870006500816080936500599A80E189B988E1CB
:10F880008AB900001A9A0A9961C240E05F9BFECFD4
:10F890008CB19927182F242F33272330310551F1AC
:10F8A000243031054CF421303105B9F022303105D6
:10F8B000E4F4232B61F04FC02530310561F1253090
:10F8C0003105F4F02630310509F442C044C08B31D3
:10F8D00009F041C041E0082FD9CF813011F08315E4
:10F8E000A1F6382E42E00827D1CF9927B82EAA24B6
:10F8F00043E004C09927A82AB92A44E00127C6CFCB
:10F900008E3019F645E00827C25EDE4F1982188254
:10F91000CE51D140BBCFC25EDE4FE881F981CE51DE
:10F92000D140EC0FFD1F8183C25EDE4F28813981FB
:10F93000CE51D1402F5F3F4FC25EDE4F39832883C7
:10F94000CE51D14008272A153B0529F446E09ECF29
:10F95000801721F09ACF473009F098CFE9818E2F98
:10F9600099278331910509F409C184319105F4F493
:10F970008630910509F4D6C0873091057CF4823039
:10F98000910509F46BC18330910524F4019709F4C2
:10F9900048C0A9C1039709F45BC0A5C18031910596
:10F9A0000CF4A1C142970CF459C1B8C0883191053B
:10F9B00009F480C08931910564F48531910509F419
:10F9C000DDC0853191050CF44EC1469709F44BC159
:10F9D0008AC18A31910509F462C08A3191050CF41B
:10F9E0008AC08B31910509F44FC04D9709F07BC156
:10F9F0009D81903359F48F81882311F48EE107C0E3
:10FA0000813011F487E903C082E001C080E017E093
:10FA1000A12EB12C1A821B829C831D828E831F8291
:10FA200067C1BBE0AB2EB12C1A8288E08B8381E4E6
:10FA30008C8386E58D8382E58E8389E48F8383E5DD
:10FA4000888780E589878FE58A8782E38B8750C125
:10FA50008A8199278039910551F0813991056CF09F
:10FA60008139910531F08239910529F006C08FE086
:10FA700005C082E003C08AE001C080E0A3E0AA2EB6
:10FA8000B12C1A828B8334C18D81882311F48EE1CD
:10FA90002BC0813011F487E927C082E025C0F4E053
:10FAA000AF2EB12C1A8289E0E1E0F0E0809368008B
:10FAB00084911EC08B81803589F48C81883039F423
:10FAC00089E0E2E0F0E08093680084910DC089E075
:10FAD000E0E0F0E080936800849106C089E0E3E014
:10FAE000F0E0809368008491E4E0AE2EB12C1A829D
:10FAF0008B831C82FDC08D81836C99E0E1E0F0E096
:10FB0000082E90936800E8958091680080FDFCCFF6
:10FB100073E0A72EB12C1A821B82EAC0442455241C
:10FB200032019CC08A819927AA27BB27F82EEE2490
:10FB3000DD24CC248B819927AA27BB27DC019927B8
:10FB40008827C82AD92AEA2AFB2A8C819927AA273A
:10FB5000BB27BA2FA92F982F8827C82AD92AEA2A83
:10FB6000FB2A8D819927AA27BB27C82AD92AEA2AE6
:10FB7000FB2ACC0CDD1CEE1CFF1C70C08A8199276F
:10FB8000582F44278B819927482B592BBE01655F3D
:10FB90007F4F46015701E33109F04AC030E0431678
:10FBA00038EF530631E0630630E0730698F483E0E3
:10FBB000F20160925B0080936800E8958091680094
:10FBC00080FDFCCF80E091E0A0E0B0E0480E591E3F
:10FBD0006A1E7B1EA1E0FB0121918191BF01992743
:10FBE000982F88273327822B932B0C01F601E09264
:10FBF0005B00A0936800E895112402E010E020E08B
:10FC000030E0C00ED11EE21EF31E4250504019F7E4
:10FC100085E0F401A0925B0080936800E8958091F4
:10FC2000680080FDFCCF81E180936800E89516C0F4
:10FC3000CEBABB27AF2D9E2D8D2D8FBB0894C11C36
:10FC4000D11CE11CF11CDB018D91BD018DBBE29A41
:10FC5000E19AE199FECF4150504051F7B2E0AB2E0E
:10FC6000B12C1A8245C08A819927382F22278B818F
:10FC70009927282B392BF3E0AF2EB12CA20EB31EFF
:10FC80001A82AE014D5F5F4FE431B9F4EBBEF6016D
:10FC900087919691FA018193892F9927DF018D939E
:10FCA000AD0182E090E0A0E0B0E0C80ED91EEA1EEF
:10FCB000FB1E2250304051F713C0CEBABB27AF2DE8
:10FCC0009E2D8D2D8FBB0894C11CD11CE11CF11CF5
:10FCD000E09A8DB3DA018D93AD012150304069F780
:10FCE000FA01108205C092E0A92EB12C80EC8A8323
:10FCF0008BE10E941AFC0BE1832D0E941AFC032564
:10FD00008B2D9927182F0E941AFC01278A2D0E94FB
:10FD10001AFC0A258EE00E941AFC8EE008274E018C
:10FD20000894811C911CA114B10459F0D4011D91B7
:10FD30004D01812F0E941AFC01270894A108B108E7
:10FD4000F2CF802F0E941AFC33949FCD80916400E3
:10FD50008E7F80936400809165008E7F8093650024
:10FD600084E690E00E9403FC0000599881E18093B2
:0CFD70006800E8951F921F920895FFCFD5
:040000031000F800F1
:00000001FF
